:020000040000FA
:10000000002905110508A500A50CA50CA50C0730B5
:10001000A505051538300505A5048501080008303B
:10002000A900AA01AB01AC0109302505031D1A285E
:1000300029151E28251CA914A51D291412302505D3
:10004000031935282208A51CAA07251A2928AA025F
:10005000291624302505031908002208A51EAB0720
:1000600025190800AB02A91608000230A006A01C42
:10007000080024302505031908000130A51EAC0234
:1000800025190800AC070800AE00AF002111A1112E
:10009000851C4828EC21851C4828051C8228B101B4
:1000A0000830B00000306820851C8428E3202E082A
:1000B000B1066820851C8428AE0CB00B5728310986
:1000C0006820851C8428E32001306820DC2008009B
:1000D00001398316031D0514031905108312073017
:1000E000A700A70B71288316851083120F30A70075
:1000F000A70B78288316851483120130A700A70B5D
:100100007F28080021150800831605148514831222
:10011000A11508002110A11005188C286430A80032
:1001200085189628E320A80B9028D8280830B0001E
:10013000B101DE20C320851CD8280310AD0CAD040E
:10014000B106B00B9A28C320851CD828B106E3203D
:10015000C320851CD828003A0319B1010319A82827
:10016000831605108312E020831685108312DC208D
:10017000831685148312E020831605148312B11FA1
:10018000DA28DC2008000330A700A70BC528831657
:10019000851083120F30A700A70BCC288316851477
:1001A00083120730A700A70BD3280518803400342A
:1001B00021140800A11408000830ED290330ED29AE
:1001C000E128E22800000000080082079029932916
:1001D0007F299629A629A429BC29D429AC29D42968
:1001E000A929D429BE298729C629C929CC29D429D6
:1001F000D429D429D429D429D429D42977297D29CB
:10020000FF2383169000873081008B019F013B30D4
:10021000850083120730990000308500D921013014
:10022000A2003F30A400A301AA30B6000030B700FE
:100230000230B500E0215829051C6429C8300102AC
:10024000031C1C2981010120201B1C29A01E1C2924
:10025000250936390319A301240825060939B200F6
:1002600025093639320403191C2924082504363A95
:100270003639031D3D29A30141290C302302031CFB
:10028000A30A03302302031C0030A2000230A2079D
:100290002508A4000F202908B6002A08B7002B085B
:1002A000B8000330A11F57292C08B9000430B5004D
:1002B000363084000008442021196429A1195A29E4
:1002C000840AB50B5A291C298A20A118CF29211884
:1002D0001C29211A8229A11A8A29E6302D02031825
:1002E000E528D429FA304420A119722908002F08E2
:1002F000FA3A031D5A2972211C2972210E297221F2
:1003000021161C2972212D08B40021121C297221EA
:10031000A1161C297221F2212D08B300A1121C295B
:10032000722120121C29722120161C2972212008FA
:10033000B600A9183614291836153408B700330842
:10034000B8000330B50058297221412972212013C9
:100350001C29722120171C2972210518AD298A2019
:100360002118AD292D08FF3A0319BC29133A0319A6
:10037000BC29EC3A4420AD2972211C29722100309D
:10038000A11B0330B6000130B50058297221A01618
:100390001C297221A0121C297221D9211C29FE308E
:1003A0004420A119CF291C29FC304420A119D429AB
:1003B0001C296430B3000230B400A001A101080080
:1003C000C830A800FA30A7000000E629E729A70BEB
:1003D000E429A80BE22908001930A7000000A70BA8
:1003E000EE290800A11B0800211FFE2950302D0610
:1003F000031DFC29A117080021130800C83033068B
:10040000031D080064302D06031D08002117080095
:100410004234593420344A344A3431344F34443429
:020420004D3459
:02400E00C43FAD
:00000001FF
